:100000000C9421050C9469050C9469050C94690500
:100010000C9469050C9469050C9469050C946905A8
:100020000C9469050C9469050C9469050C943110C5
:100030000C9469050C94301E0C9469050C946905A8
:100040000C9469050C9469050C9469050C94891E3F
:100050000C9469050C9469050C9469050C94690568
:100060000C9469050C9469050C9469050C94690558
:100070000C946905970EBE0EB60FBE0EB60F0A0F92
:100080002D0FB60F840F930F661466149E149E14E2
:1000900019154D154417441764154417F514F51434
:1000A000FE16441713173117804E4C31302F0C12A7
:1000B00013508062635880514F595C5E5B66525AA0
:1000C0005D4B492A2E2D2526275F606157565354D4
:1000D00055802834330F3637381D1B06190510118B
:1000E0002C041607090A0E0D0B2B141A0815181CE0
:1000F00017351E1F20212423227C78657B7D7939CA
:100100004A808080808080805B20723D2530346C06
:1001100058206B6579636F64653D253032582070D7
:100120007265737365643D2558204354524C3D25D8
:10013000582053484946545F4C4546543D25582065
:1001400053484946545F524748543D255820434D33
:10015000445F4C4546543D255820434D445F52472B
:1001600048543D255820414C545F4C4546543D254C
:100170005820414C545F524748543D2558205D0A51
:1001800000506F77657220737461746520300A00C7
:10019000506F77657220737461746520310A005B5B
:1001A000204E655854206B6579626F6172642069D6
:1001B0006E697469616C697A6564205D0A00496ED4
:1001C000697469616C20706F7765722062757474F0
:1001D0006F6E2073746174653A2025620A005B209B
:1001E000496E7469616C697A696E67204E6558540E
:1001F000206B6579626F617264205D0A000A4C6F42
:100200006F702073746172742E0A000A5553422075
:10021000636F6E666967757265642E0A000A544DD5
:100220004B3A3937346337382F4C5546413A6436A8
:10023000613764660A003E034E00650058005400B2
:1002400020004B006500790062006F0061007200C1
:100250006400200074006F0020005500530042002D
:10026000200063006F006E0076006500720074006D
:100270006500720000000E0374002E006D002E0059
:100280006B002E000000040309040902540003015E
:1002900000A032090400000103010100092111013D
:1002A00000012240000705810308000A090401003B
:1002B0000103010200092111010001227F0007054D
:1002C0008203080001090402000103000000092163
:1002D0001101000122220007058303200001120101
:1002E000100100000008EDFEBCBC00050102000189
:1002F0000631FF0974A1010975150026FF0095203C
:10030000750881020976150026FF00952075089171
:1003100002C005010902A1010901A1008501050929
:1003200019012908150025019508750181020501AB
:10033000093009311581257F950275088106093834
:100340001581257F950175088106050C0A3802156F
:1003500081257F950175088106C0C005010980A12E
:100360000185021601002637001A81002AB70075A0
:100370001095018100C0050C0901A101850316013A
:1003800000269C021A01002A9C027510950181002A
:10039000C005010906A101050719E029E715002597
:1003A00001950875018102950175088101050819FB
:1003B00001290595057501910295017503910105C6
:1003C00007190029FF150026FF0095067508810012
:1003D000C0636F6E73756D65723A20253034580AAC
:1003E0000073797374656D3A20253034580A000A19
:1003F000002530325820006B6579626F6172643A73
:1004000020004C45443A20253032580A0025583AFD
:100410002530386225730A000A2020303132333407
:100420003536370A00290A002575002F002575008A
:100430005D2800256400200025640020002564005C
:1004400020002564007C0025303258006D6F7573E4
:10045000656B6579205B62746E7C782079207620EC
:10046000685D287265702F61636C293A205B006DAE
:100470006B5F776865656C5F74696D655F746F5FEE
:100480006D6178203D2025640A006D6B5F7768659B
:10049000656C5F6D61785F7370656564203D2025D4
:1004A000640A006D6B5F74696D655F746F5F6D6189
:1004B00078203D2025640A006D6B5F6D61785F7365
:1004C00070656564203D2025640A006D6B5F696E70
:1004D00074657276616C203D2025640A006D6B5F47
:1004E00064656C6179203D2025640A006D6B5F773F
:1004F0006865656C5F74696D655F746F5F6D617869
:10050000203D2025640A006D6B5F776865656C5F30
:100510006D61785F7370656564203D2025640A0015
:100520006D6B5F74696D655F746F5F6D6178203DA1
:100530002025640A006D6B5F6D61785F737065657F
:1005400064203D2025640A006D6B5F696E746572DE
:1005500076616C203D2025640A006D6B5F64656CDC
:100560006179203D2025640A000A00257500363A8D
:1005700020776865656C5F74696D655F746F5F6D2A
:1005800061783A20000A00257500353A20776865C1
:10059000656C5F6D61785F73706565643A20000A11
:1005A00000257500343A2074696D655F746F5F6D66
:1005B00061783A20000A00257500333A206D617891
:1005C0005F73706565643A20000A00257500323A51
:1005D00020696E74657276616C286D73293A20000B
:1005E0000A00257500313A2064656C6179282A314A
:1005F000306D73293A20000A092D2056616C75650B
:1006000073202D0A004D3E004D25643E20003F0022
:100610007365742064656661756C740A00433E20DE
:100620000077686572652064656C74613A20637553
:1006300072736F723D25642C20776865656C3D256B
:10064000640A53656520687474703A2F2F656E2EA6
:1006500077696B6970656469612E6F72672F77695E
:100660006B692F4D6F7573655F6B6579730A000A4F
:10067000092D204D6F7573656B6579202D0A4553E3
:10068000432F713A09717569740A313A0964656CCE
:100690006179282A31306D73290A323A09696E74FA
:1006A000657276616C286D73290A333A096D617839
:1006B0005F73706565640A343A0974696D655F74C7
:1006C0006F5F6D61780A353A09776865656C5F6DB3
:1006D00061785F73706565640A363A0977686565A5
:1006E0006C5F74696D655F746F5F6D61780A0A7025
:1006F0003A097072696E742076616C7565730A646C
:100700003A097365742064656661756C74730A7563
:10071000703A092B310A646F776E3A092D310A70ED
:100720006775703A092B31300A7067646F776E3ADB
:10073000092D31300A0A7370656564203D206465B7
:100740006C7461202A206D61785F73706565642028
:100750002A2028726570656174202F2074696D6588
:100760005F746F5F6D6178290A003F004D3E200085
:10077000433E20004C25640A000A092D20436F6E79
:10078000736F6C65202D0A4553432F713A097175BB
:1007900069740A6D3A096D6F7573656B65790A0046
:1007A0000A092D204D61676963202D0A643A0964A6
:1007B000656275670A783A096465627567206D61DC
:1007C000747269780A6B3A096465627567206B65B3
:1007D00079626F6172640A6D3A09646562756720B7
:1007E0006D6F7573650A763A0976657273696F6E17
:1007F0000A733A097374617475730A633A09636F13
:100800006E736F6C65206D6F64650A302D343A0924
:100810006C61796572302D34284631302D4634298B
:100820000A506175733A09626F6F746C6F61646529
:10083000720A003F0074696D65725F7265616433AE
:100840003228293A202530346C580A006B657962C9
:100850006F6172645F69646C653A2025580A006BA9
:100860006579626F6172645F70726F746F636F6CD1
:100870003A2025580A00686F73745F6B6579626F60
:100880006172645F6C65647328293A2025580A00F8
:100890000A092D20537461747573202D0A00474393
:1008A000433A20352E342E30204156522D4C4942A9
:1008B000433A20322E302E30204156525F4152436F
:1008C000483A2061767233350A004F5054494F4EF2
:1008D000533A204C554641204D4F5553454B4559B1
:1008E0002045585452414B455920434F4E534F4C8D
:1008F0004520434F4D4D414E44204B45594D4150AD
:100900005F53454354494F4E20343039360A004234
:1009100055494C443A203937346337382028303829
:100920003A33343A30392041707220313720323036
:100930003232290A005649443A2030784645454427
:1009400028742E6D2E6B2E29205049443A20307881
:1009500042434243284E655854204B6579626F618B
:10096000726420746F2055534220636F6E766572F7
:1009700074657229205645523A203078303530302F
:100980000A00444553433A2055534220636F6E7624
:10099000657274657220666F72204E655854206EC1
:1009A0006F6E2D414442204B6579626F6172640A1B
:1009B000000A092D2056657273696F6E202D0A009A
:1009C0000A6D6F7573653A206F66660A000A6D6F6F
:1009D0007573653A206F6E0A000A6B6579626F6104
:1009E00072643A206F66660A000A6B6579626F610D
:1009F00072643A206F6E0A000A6D61747269783A07
:100A0000206F66660A000A6D61747269783A206F19
:100A10006E0A000A64656275673A206F6E0A000A02
:100A200064656275673A206F66660A000A0A626F3B
:100A30006F746C6F616465722E2E2E2000433E2011
:100A4000000011241FBECFEFD4E0DEBFCDBF04B63F
:100A500003FE28C080912C0390912D03A0912E03BA
:100A6000B0912F038730904BA740B04BD9F4109230
:100A70002C0310922D0310922E0310922F0314BEFC
:100A80000FB6F894A895809160008861809360000B
:100A9000109260000FBE1092010810920008E0E072
:100AA000F8E3099511E0A0E0B1E0ECE2FEE402C059
:100AB00005900D92A433B107D9F723E0A4E3B1E088
:100AC00001C01D92AC32B207E1F70E94B00B0C944A
:100AD00014270C940000FF93EF93E0913401F09100
:100AE0003501309709F00995EF91FF910895FC01C8
:100AF0008591803011F0EFDFFBCF0895FF27E0E212
:100B000030E247FF0CC0419597FF09C0EDE26095C8
:100B1000709580959095611D711D811D911D27FF18
:100B200002C0219530E350E2AA27660F771F881F85
:100B3000991FAA1FA41710F0A41B63955A95A9F733
:100B4000AA3008F0A95FA05DAF93F3956115710518
:100B50008105910541F7ED3211F4EF93F395F2170A
:100B600018F43F93F395FBCF8F91B5DFFA95E1F73A
:100B70000895E991F9918591803021F0853219F03D
:100B8000AADFF9CF089520E0E89455915532C1F3DA
:100B9000503311F4689455915A3348F4505390F3FC
:100BA000220F022E220F220F200D250FF4CF0EF45C
:100BB000219589919991533619F3533729F153357A
:100BC00059F1BC0188279927E8945C3621F4899172
:100BD000999168945591543639F446EF7EF077FF39
:100BE0000DC08FEF9FEF0AC055374AE039F05835F6
:100BF00040E121F0523642E009F00895FF93EF936F
:100C00007DDFEF91FF91B7CFFF93EF93FC018191CF
:100C10008030B9F360DFFBCFFF93EF9368DFF1CF54
:100C2000DF93CF93CDB7DEB72596A3DFCF91DF91CA
:100C30000895CF93DF93D82FD770E82FE695E695E8
:100C4000E695CE2FCF706D2F8C2F0E9474128111DC
:100C500010C0EC2FF0E0E95CFE4F81E090E001C0B5
:100C6000880FDA95EAF79081892B808381E0809361
:100C70003601DF91CF910895CF93DF93D82FD770AE
:100C8000E82FE695E695E695CE2FCF706D2F8C2F49
:100C90000E947412882389F0EC2FF0E0E95CFE4F8B
:100CA00081E090E001C0880FDA95EAF780959081A5
:100CB0008923808381E080933601DF91CF9108956D
:100CC00080910E03816080930E032FEF84E39CE0FC
:100CD000215080409040E1F700C0000080910E0359
:100CE00080FF08C08EED91E09F938F930E941006C5
:100CF0000F900F90569A5E9A54984C9A89B19091A1
:100D00000E0390FF11C082958F7091E0892781704A
:100D10001F928F938EEB91E09F938F930E9410060A
:100D20000F900F900F900F900E942C08E7E3F1E0D6
:100D3000119221E0E334F207D9F780910E0380FF8E
:100D400008C08FE991E09F938F930E9410060F9047
:100D50000F9008954F925F926F927F928F929F9221
:100D6000AF92BF92CF92DF92EF92FF928FE19EE41B
:100D70000197F1F700C000005E981092360188E5F7
:100D80004C990DC00E941906809136018823C9F044
:100D900080910E0380FF15C080E991E00CC00E9495
:100DA0003C0680913601882361F080910E0380FF1C
:100DB00008C081E891E09F938F930E9410060F90E6
:100DC0000F900E9496086B017C01672B682B692BA2
:100DD00009F4DBC0C11496E0D90690E3E906F104FA
:100DE00009F4D3C05E9A80910E0326013701442492
:100DF0009FE0592266247724460157019924AA24AA
:100E0000BB2480FF77C0D701C60142E1B695A79504
:100E1000979587954A95D1F7817099279F938F93DE
:100E2000D701C60151E1B695A795979587955A9533
:100E3000D1F7817099279F938F93C701817099276C
:100E40009F938F93D701C6016FE0B695A7959795AD
:100E500087956A95D1F7817099279F938F93D701D2
:100E6000C6017EE0B695A795979587957A95D1F7B7
:100E7000817099279F938F93D701C601EDE0B695B6
:100E8000A79597958795EA95D1F7817099279F93B4
:100E90008F93D701C601FCE0B695A79597958795E6
:100EA000FA95D1F7817099279F938F9381E0411430
:100EB00094E059066104710409F080E01F928F9359
:100EC000D501C401B695A795979587959F938F9364
:100ED000FF92EF92DF92CF9288E091E09F938F9301
:100EE0000E9410068DB79EB748960FB6F8949EBF25
:100EF0000FBE8DBF81E5E2FE03C00E94190602C04D
:100F00000E943C0682E5E1FE03C00E94190602C071
:100F10000E943C0683E5E0FE03C00E94190602C061
:100F20000E943C0684E5D7FE03C00E94190602C059
:100F30000E943C0685E5D6FE03C00E94190602C049
:100F40000E943C0686E5D5FE03C00E94190602C039
:100F50000E943C0687E5D4FE03C00E94190602C029
:100F60000E943C06D501C401B695A7959795879533
:100F7000411494E059066104710419F40E941906A1
:100F800002C00E943C0681E001C080E0FF90EF902B
:100F9000DF90CF90BF90AF909F908F907F906F9099
:100FA0005F904F900895E82FF0E0E95CFE4F80815C
:100FB000089581FF03C061E081E002C060E080E04D
:100FC0000C9451085998519A08955198599A089536
:100FD0000E94E2078FE094E00197F1F700C0000063
:100FE0000E94E5078FEC90E00197F1F700C0000048
:100FF0000E94E2078FE692E00197F1F700C000003F
:101000000C94E5070E94E2078FEC90E00197F1F75E
:1010100000C000000E94E5078FE393E00197F1F71D
:1010200000C000000E94E2078FEC90E00197F1F70A
:1010300000C000000E94E5078FED94E00197F1F7F2
:1010400000C000000E94E2078FE198E00197F1F7ED
:1010500000C000000C94E5070E94E5075098589ADC
:101060000E94E8078FE094E00197F1F700C00000CC
:101070000E9402088FE796E00197F1F700C0000098
:101080000E94E8078FE094E00197F1F700C00000AC
:101090000E9402088FE796E00197F1F700C0000078
:1010A0000895CF93DF93D82FC62FF8940E94E207BC
:1010B0008FE497E00197F1F700C000000E94E50778
:1010C0008FE692E00197F1F700C000000E94E2076E
:1010D0008FEC90E00197F1F700C00000DD2319F0DC
:1010E0000E94E50702C00E94E2078FEC90E00197A2
:1010F000F1F700C00000CC2319F00E94E50702C000
:101100000E94E2078FEC90E00197F1F700C0000029
:101110000E94E2078FEA95E00197F1F700C0000016
:101120000E94E5077894DF91CF910895489B13C002
:101130000E94E807F89480E593EC489B08C000976C
:1011400041F025E02A95F1F700000197F6CF892BB1
:1011500041F40E940208789430E020E080E090E0C2
:101160001AC085E88A95F1F7000086E140E050E07A
:10117000BA01489960647695679557954795EFEC65
:10118000F0E03197F1F700C00000815091F77894BA
:10119000342F252FCB01632F722F089580914E029B
:1011A0000895CF93DF9300D01F92CDB7DEB7209183
:1011B0002303243021F523E029839B838A8382E063
:1011C0008093E9008FEF9091E800815095FD06C073
:1011D00095ED9A95F1F700008111F5CF8091E80027
:1011E00085FF0DC040E050E063E070E0CE01019665
:1011F0000E94680D8091E8008E778093E8000F9040
:101200000F900F90DF91CF910895CF93DF9300D08F
:101210001F92CDB7DEB720912303243061F51982E8
:101220001A821B8222E029838138910520F08058A0
:1012300091099B838A8382E08093E9008FEF9091EC
:10124000E800815095FD06C095ED9A95F1F70000F4
:101250008111F5CF8091E80085FF0DC040E050E09E
:1012600063E070E0CE0101960E94680D8091E80075
:101270008E778093E8000F900F900F90DF91CF91C1
:10128000089520912303243051F522E02093E900B2
:101290002FEF3091E800215035FD06C035ED3A952D
:1012A000F1F700002111F5CF2091E80025FF17C0CC
:1012B00020911001222341F021E02093F10040E031
:1012C00050E065E070E004C040E050E063E070E0B2
:1012D0000E94680D8091E8008E778093E800089561
:1012E000CF93DF9320912303243049F521E020930D
:1012F000E90021E8215059F03091E80035FD07C0A0
:10130000EFE3F1E03197F1F700C00000F3CF209157
:10131000E80025FF14C0EC0140E050E068E070E018
:101320000E94680D8091E8008E778093E80088E045
:10133000FE01A6E4B2E001900D928A95E1F7DF91FB
:10134000CF910895CF93C0914501C1110BC00E9468
:101350006E1E643C79408105910520F081E0809308
:101360004501C1E08C2FCF910895FF920F931F93F9
:10137000CF93DF93D82F0FB607FE83C0809123034E
:10138000843081F08091030190E001962091050165
:1013900030E0822393232091040130E082179307E9
:1013A00009F0C9C00E94A209811110C080910301F7
:1013B00090E001962091050130E082239323209153
:1013C000040130E08217930709F0B5C00E94621E45
:1013D0008C01C091E900CF709091EC00892F817051
:1013E00090FD80E8C82B83E08093E90085E0F82E2B
:1013F0008091EB0085FD42C08091EB0080FF3EC0F4
:101400008091EE0087FF3AC0809104019091030122
:10141000981709F457C09091E80095FF8AC0E091B1
:101420000101F0910201E80FF11D20818F5F909181
:1014300005018923809304012093F1008091E80045
:1014400085FDE2CF8091E80080FFDECF8091E8004B
:101450008E778093E800F0920001D6CF809103014F
:1014600090E001962091050130E0822393232091A2
:10147000040130E08217930709F448C0CF70C0938D
:10148000E90040910301842F90E00196209105012D
:1014900030E0822393232091040130E082179307E8
:1014A00009F44CC0E0910101F0910201E40FF11D3B
:1014B000D083809103018F5F9091050189238093F0
:1014C00003013CC08091E80085FF33C0D093F10058
:1014D00081E09091F200992391F09091E80090FFC3
:1014E0000EC09091E80095FF03C01092F100F9CF73
:1014F0009091E8009E779093E800F0920001882395
:1015000009F4ACCFCF70C093E90018C080910001FE
:10151000882309F4B3CF0E94621E9C0180179107B3
:1015200011F4890165CF90910001915090930001D1
:10153000F8CF80E0CECF40910301B4CF80E0DF91BF
:10154000CF911F910F91FF900895809122038111F7
:1015500004C00E94CE0F0C94211008951092220313
:101560000895089542E061EC81E00E94E10C42E0C0
:1015700061EC82E00E94E10C46E261EC83E00C94B5
:10158000E10C80912503833009F453C030F481309D
:1015900071F0823009F4BAC008958A3009F4A6C007
:1015A0008B3009F478C0893009F0C8C020C0809120
:1015B0002403813A09F0C2C08091E800877F8093BC
:1015C000E8008091280390912903892B21F468E099
:1015D00086E492E003C060E080E090E070E00E946A
:1015E000B50D8091E8008B778093E8000895809195
:1015F0002403813209F0A2C080912803909129032D
:10160000892B09F09BC08091E800877F8093E800D8
:101610008091E80082FD05C0809123038111F8CFFD
:101620008DC08091F10080934E028091E8008B770D
:1016300081C080912403813A09F080C08091280301
:1016400090912903892BA1F48091E800877F8093F2
:10165000E8008091E80080FFFCCF80911101809329
:10166000F1008091E8008E778093E8000E94160DCB
:101670008091280390912903019709F05FC0809120
:10168000E800877F8093E8008091E80080FFFCCF2E
:10169000809110014AC080912403813209F04EC02C
:1016A0008091280390912903892B69F48091E800A7
:1016B000877F8093E8000E94160D80912603809317
:1016C00011010E941614809128039091290301971B
:1016D000A9F58091E800877F8093E8000E94160DAD
:1016E00080912603809310010C941614809124039A
:1016F000813221F58091E800877F8093E8000E9485
:10170000160D8091270380934F0208958091240342
:10171000813AA1F48091E800877F8093E80080916E
:10172000E80080FFFCCF80914F028093F100809110
:10173000E8008E778093E8000C94160D08950E94BF
:10174000F31D80912103882329F00E941C1E811122
:101750000C94CB0C089508950C94AB0B0C94AB0B2C
:10176000CF9384B7877F84BF0FB6F894A8958091F4
:101770006000886180936000109260000FBE90E06E
:1017800080E80FB6F89480936100909361000FBEDB
:1017900085EB99E00E94C51D86E091E00E94F6105D
:1017A0008DE192E00E9477050E94AE0B0E94C81165
:1017B0000E94CE0F0E94211078940E94CA1180913D
:1017C0002303843029F00E94DB100E94AB0BF7CF7B
:1017D0000E94A2098823B9F38BE092E00E9477056A
:1017E0000E94AC0B8DEF91E00E947705C3E08091E1
:1017F0002303853019F40E949F0BF9CF0E94DC1D52
:101800000E94CE112091E4003091E50080914301C7
:10181000909144012817390709F464C08091E400CD
:101820009091E50090934401809343010E94A209A6
:10183000882309F457C080912303843009F052C0F3
:101840008091E9008F702091EC00922F917020FD23
:1018500090E8892BC093E9009091EB0090FF3FC086
:101860009091EE0097FF3BC09091040120910301FD
:10187000291709F12091E80025FF1DC0E091010121
:10188000F0910201E90FF11D30819F5F2091050168
:101890009223909304013093F1009091E80095FD1C
:1018A000E3CF9091E80090FFDFCF9091E8009E7722
:1018B0009093E800D9CF9091F200992381F0909114
:1018C000E80090FF0CC09091E80095FF03C01092D3
:1018D000F100F9CF9091E8009E779093E8008F7027
:1018E0008093E9000E94DB1082CF292F3327233019
:1018F0003105C9F060F42130310581F02230310525
:1019000009F041C084E590E02AE832E040C021328D
:101910003105E1F02232310531F135C082E190E04C
:101920002EED32E034C099278130910549F028F03E
:10193000029749F5E6E3F2E005C0E6E8F2E002C00E
:10194000E6E7F2E0849190E09F0121C063307105E9
:10195000D0F4660F771FFB01ED5DFE4F20813181D2
:1019600089E090E014C06330710568F4FB01EE0F6C
:10197000FF1FE35EFE4F20813181FB01E65EFE4FDB
:10198000808190E004C080E090E020E030E0FA0147
:1019900031832083089584E089BD86E089BD09B440
:1019A00000FEFDCF8091D8008F7D8093D80080917C
:1019B000E00082608093E0008091E00081FDFCCF38
:1019C0000895982F953068F59093E900981739F0AD
:1019D0007091EC002091ED005091F00003C0242F95
:1019E000762F50E021FD02C09F5FECCF3091EB00DD
:1019F0003E7F3093EB003091ED003D7F3093ED0062
:101A00003091EB0031603093EB007093EC00209349
:101A1000ED005093F0002091EE0027FDE5CF80E02F
:101A200008958F708093E90081E0089580912403E8
:101A300087FF11C08091E80082FD05C080912303DB
:101A40008111F8CF11C08091E8008B770BC0809195
:101A50002303882349F08091E80080FFF8CF80912C
:101A6000E8008E778093E80008952091E40030919B
:101A7000E50095E64091EC00842F817040FF23C083
:101A80008091E80080FD1DC080912303882399F098
:101A9000853099F08091EB0085FD11C04091E40004
:101AA0005091E5002417350729F3915011F09A0160
:101AB000E1CF84E0089582E0089583E0089581E015
:101AC000089580E008954091E80042FFDDCF089539
:101AD000CF92DF92EF92FF920F931F93CF93DF93FA
:101AE000EC018B017A010E94350D811135C0E114A2
:101AF000F10439F0F70180819181081B190BC80F9F
:101B0000D91FC12CD12C0115110529F18091E800B4
:101B100085FD18C08091E8008E778093E8000E94D0
:101B2000DB10E114F10449F0F70180819181C80EC6
:101B3000D91ED182C08285E00FC00E94350D882356
:101B400011F30AC089918093F10001501109FFEF50
:101B5000CF1ADF0AD8CF80E0DF91CF911F910F918C
:101B6000FF90EF90DF90CF90089520912A0330915D
:101B70002B032617370748F06115710539F42091BA
:101B8000E8002E772093E80001C0B901FC0120E0B5
:101B90006115710561F1809123038823D9F18530A6
:101BA000D9F18091E80083FD39C08091E80082FD81
:101BB0002BC08091E80080FFEBCF8091F20090E095
:101BC0006115710551F08830910538F42191209309
:101BD000F100615071090196F3CF21E0089709F0F7
:101BE00020E08091E8008E778093E800D1CF21112A
:101BF000D2CF0AC080912303882361F0853061F041
:101C00008091E80083FD0AC08091E80082FFF2CF56
:101C100080E0089582E0089583E0089581E00895CA
:101C200020912A0330912B032617370748F06115BE
:101C3000710539F42091E8002E772093E80001C067
:101C4000B901FC0120E06115710579F18091230350
:101C5000882309F43DC0853009F43CC08091E80038
:101C600083FD3AC08091E80082FD2CC08091E8009D
:101C700080FFE9CF8091F20090E06115710559F085
:101C80008830910540F424912093F1003196615001
:101C900071090196F2CF21E0089709F020E08091C8
:101CA000E8008E778093E800CECF2111CFCF0AC015
:101CB00080912303882361F0853061F08091E800F2
:101CC00083FD0AC08091E80082FFF2CF80E0089592
:101CD00082E0089583E0089581E008951F93CF93F3
:101CE000DF93CDB7DEB7AA970FB6F894DEBF0FBE6D
:101CF000CDBFE4E2F3E08091F100819323E0EC3288
:101D0000F207C9F70E94C10A8091E80083FF2EC143
:101D10008091240390912503492F50E04A305105CA
:101D200008F024C1FA01E65CFF4F0C94FA268038D3
:101D300021F0823809F01AC108C0809120039091E7
:101D40002103992389F082600FC0809128038F704E
:101D5000853008F00BC18093E9008091EB0085FB92
:101D6000882780F91092E9009091E800977F90937E
:101D7000E8008093F1001092F100D1C0282F2D7F50
:101D800009F0F4C0882319F0823061F0EFC080912F
:101D90002603813009F0EAC0933009F080E0809397
:101DA00021032EC08091260381112AC0809128032F
:101DB0008F702FEF280F243008F0D8C08093E900EF
:101DC0002091EB0020FF1CC0933021F48091EB00A8
:101DD000806214C09091EB0090619093EB0021E041
:101DE00030E0A90102C0440F551F8A95E2F74093E5
:101DF000EA001092EA008091EB0088608093EB008B
:101E00001092E9008091E800877F8093E8000E94AB
:101E1000160DACC08111AAC0109126031F778091C6
:101E2000E3008078812B8093E3008091E800877F36
:101E30008093E8000E94160D8091E80080FFFCCF9F
:101E40008091E30080688093E300111102C082E07A
:101E500001C083E08093230389C08058823008F05A
:101E600085C080912603909127038C3D53E0950710
:101E700079F583E08A838AE289834FB7F894DE019B
:101E8000139620E03EE051E2E32FF0E0509357003C
:101E9000E49120FF03C0E295EF703F5FEF708E2F5B
:101EA00090E0EA3010F0C79601C0C0968D939D93E4
:101EB0002F5F243149F74FBF8091E800877F8093DF
:101EC000E8006AE270E0CE0101960E94B50D16C0EE
:101ED0006091280370912903AE014F5F5F4F0E940C
:101EE000750CBC01892B09F441C09091E800977FE3
:101EF0009093E80089819A810E94100E8091E800F9
:101F00008B778093E80032C0803881F58091E800BB
:101F1000877F8093E80080911F038093F100809178
:101F2000E8008E7772CF811121C0809126039091B5
:101F3000270399270297D4F48091E800877F809344
:101F4000E8008091260380931F030E94160D809164
:101F50001F03811106C08091E30087FD02C081E06C
:101F600001C084E0809323030E94B20A8091E800BC
:101F700083FF0AC08091E800877F8093E80080910A
:101F8000EB0080628093EB00AA960FB6F894DEBF58
:101F90000FBECDBFDF91CF911F9108950E942B10EE
:101FA0000E942E10E0EEF0E0808181608083E8EDF9
:101FB000F0E080818F77808319BCE3E6F0E08081D8
:101FC000816080831092220308950E942B100E944A
:101FD0002E108091D8008F778093D8008091D80000
:101FE00080688093D8008091D8008F7D8093D8003E
:101FF00084E089BD86E089BD09B400FEFDCF109262
:10200000230310921F03109221031092200342E039
:1020100060E080E00E94E10C8091E1008E7F80937F
:10202000E1008091E20081608093E2008091E20013
:1020300088608093E2008091E0008E7F8093E000D2
:102040000895E3E6F0E080818E7F808381E08093D5
:1020500022030C94E50F1092E20008951092E10023
:1020600008951F920F920FB60F9211242F933F9352
:102070004F935F936F937F938F939F93AF93BF9390
:10208000EF93FF938091E10082FF0BC08091E2000B
:1020900082FF07C08091E1008B7F8093E1000E9466
:1020A000DA108091E10080FF18C08091E20080FF8B
:1020B00014C08091E2008E7F8093E2008091E20064
:1020C00080618093E2008091D80080628093D80084
:1020D00019BC109223030E94AE0A8091E10084FF94
:1020E00030C08091E20084FF2CC084E089BD86E08E
:1020F00089BD09B400FEFDCF8091D8008F7D80930B
:10210000D8008091E1008F7E8093E1008091E20011
:102110008F7E8093E2008091E20081608093E200F4
:1021200080911F03882311F084E007C08091E300B1
:1021300087FD02C081E001C083E0809323030E94F9
:10214000A50A8091E10083FF24C08091E20083FF13
:1021500020C08091E100877F8093E10082E080933E
:10216000230310921F038091E1008E7F8093E10092
:102170008091E2008E7F8093E2008091E200806196
:102180008093E20042E060E080E00E94E10C0E9467
:10219000B10AFF91EF91BF91AF919F918F917F9184
:1021A0006F915F914F913F912F910F900FBE0F90C4
:1021B0001F9018950895CF93809123038823A1F051
:1021C000C091E900CF709091EC00892F817090FD53
:1021D00080E8C82B1092E9008091E80083FD0E94FE
:1021E0006E0ECF70C093E900CF9108959093550281
:1021F000809354020895E0915402F0915502309773
:1022000021F00190F081E02D099480E00895EF9293
:10221000FF920F931F93CF93DF93E0915402F091BD
:1022200055023097B1F18C010280F381E02D0995C0
:1022300080910E0382FF2DC080FF04C087EF93E0E2
:102240000E947705E80118E081EFE82E83E0F82E80
:1022500080910E0380FF0BC088811F928F93FF92A5
:10226000EF920E9410060F900F900F900F90115058
:1022700021961111EDCF80910E0380FF0AC08FEEE1
:1022800093E0DF91CF911F910F91FF90EF900C940D
:102290007705DF91CF911F910F91FF90EF900895F7
:1022A0001F93CF93DF932091540230915502232B3B
:1022B00089F0EC0118810E94C3219881892B8883C1
:1022C000E0915402F09155020480F581E02DCE0199
:1022D00009951883DF91CF911F910895CF93DF93D4
:1022E00020915202309153022817390709F1909337
:1022F000530280935202E0915402F09155023097BC
:10230000B9F0EC010680F781E02D099580910E036C
:1023100082FF0EC080FF0CC0DF93CF9381EE93E06D
:102320009F938F930E9410060F900F900F900F9025
:10233000DF91CF910895CF93DF9320915002309198
:1023400051022817390709F19093510280935002E6
:10235000E0915402F09155023097B9F0EC010084FD
:10236000F185E02D099580910E0382FF0EC080FF5C
:102370000CC0DF93CF9381ED93E09F938F930E94E6
:1023800010060F900F900F900F90DF91CF9108954E
:102390000C9473120E94591E0C946006BF92CF9247
:1023A000DF92EF92FF920F931F93CF93DF9300D0B2
:1023B00000D01F92CDB7DEB70E94AA0607E512E053
:1023C000F12C8F2D0E94D307B82EF801C080C826AB
:1023D00039F4F3940F5F1F4FFCE0FF12F2CF30C0CF
:1023E00080910E0381FD0E948812D12CEE24E3948B
:1023F0008C2D8E21F9F0D982FA8291E08B2D8E21DD
:1024000009F490E09B830E94621E8160782F9D8377
:102410008C8349815A816B818D810E94BE124981D2
:102420005A816B817C818D810E94DE1DF801808143
:102430008E258083D394EE0CF8E0DF12D9CFC9CF7C
:102440008FEF89838A831B820E94621E8160782FAE
:102450009D838C8349815A816B818D810E94BE123C
:102460000E94DD1D0E9411210E94FB1090915602D6
:10247000891741F10E94FB108093560290910E0340
:1024800092FF0EC090FF0CC01F928F9382E094E0E9
:102490009F938F930E9410060F900F900F900F90B4
:1024A000809156020F900F900F900F900F90DF9138
:1024B000CF911F910F91FF90EF90DF90CF90BF9041
:1024C0000C94EF1D0F900F900F900F900F90DF91D5
:1024D000CF911F910F91FF90EF90DF90CF90BF9021
:1024E00008950C94D9070895CF93C62F0E94D3075F
:1024F00021E030E002C0220F331FCA95E2F790E0DE
:102500002823392381E0232B09F480E0CF9108951B
:10251000EF92FF920F931F93CF93DF9388E194E0A4
:102520000E947705C0E0D0E089E2E82E81E0F82E35
:102530000DE014E08C2F0E94D3070E94CA1DFF9269
:10254000EF921F928F93DF93CF931F930F930E946D
:10255000100621968DB79EB708960FB6F8949EBFC9
:102560000FBE8DBFCC30D10529F7DF91CF911F91E0
:102570000F91FF90EF90089508950895CF93DF9302
:10258000CDB7DEB72B970FB6F894DEBF0FBECDBF29
:10259000942F4F83252F588769877A878B874A85A1
:1025A0005B85452B31F02F3F31F481E09F3F19F4DB
:1025B00003C081E001C080E080FD07C04F815885E5
:1025C00069857A858B850E94DE1DDE01119686E085
:1025D000FD0111928A95E9F785E0FE013796019099
:1025E0000D928A95E1F749815A816B817C818D81B9
:1025F0009E810E94331A2B960FB6F894DEBF0FBE51
:10260000CDBFDF91CF910895CF93882309F4C4C043
:10261000C82F8CEF8C0F813A48F48C2F0E943F24F6
:102620008111BAC08C2F0E94271D0CC080E28C0F34
:10263000883058F4C77081E001C0880FCA95EAF766
:102640000E94651DCF910C949F1D8BE58C0F8330EC
:1026500078F4C53A29F0C63A31F083E890E005C035
:1026600081E890E002C082E890E0CF910C946E1176
:1026700088E58C0F873108F08FC0C83A09F445C04F
:10268000C93A09F445C0CA3A09F445C0CB3A09F43D
:1026900045C0CC3A09F445C0CD3A09F445C0CE3A1C
:1026A00009F445C0CF3A09F445C0C13B09F445C01F
:1026B000C03B09F445C0C23B09F445C0C33B09F423
:1026C00045C0C43B09F445C0C53B09F445C0C63B01
:1026D00009F445C0C73B09F445C0C83B09F445C0EF
:1026E000C93B09F445C0CA3B09F445C0CB3B09F4DA
:1026F00045C0CC3B09F445C0CD3B09F445C0CE3BB9
:1027000009F445C080E090E044C082EE90E041C012
:1027100089EE90E03EC08AEE90E03BC085EB90E011
:1027200038C086EB90E035C083EB90E032C084EB9C
:1027300090E02FC087EB90E02CC08CEC90E029C09B
:102740008DEC90E026C083E891E023C08AE891E018
:1027500020C082E991E01DC084E991E01AC081E2C5
:1027600092E017C083E292E014C084E292E011C0CC
:1027700085E292E00EC086E292E00BC087E292E032
:1027800008C08AE292E005C08FE690E002C080E7D0
:1027900090E0CF910C949B11CF910895882329F15B
:1027A0009CEF980F913A18F40E94441D0DC090E2DE
:1027B000980F983058F4877091E001C0990F8A956E
:1027C000EAF7892F0E946B1D0C949F1D9BE5980FC3
:1027D000933020F480E090E00C946E11885A873199
:1027E00020F480E090E00C949B110895882321F060
:1027F0000E94651D0C949F1D0895882321F00E945E
:102800006B1D0C949F1D08950E94851D0E94541DF0
:102810000E949F1D0E94B7210E94842080E090E0CA
:102820000E946E1180E090E00C949B110E94751D37
:102830000C940414CF92DF92EF92FF920F931F93A8
:10284000CF93DF9300D000D01F92CDB7DEB76C01DD
:102850000E94F11D811118C385E0F601DE01119679
:1028600001900D928A95E1F7F60140815181238113
:1028700034812115310531F05F3F31F481E04F3F64
:1028800019F403C081E001C080E080FDFDC2F601C3
:10289000F280E580E2948FE0E82249835A83FB824C
:1028A000722F3D832C836F2D8D810E949C1C8C0187
:1028B0000E949B1C0E948B1BE12FE295EF708E2FD4
:1028C00090E0FC01EC5BFF4F0C94FA26812F807F97
:1028D0001F70882311F01295107FFF20B9F011238B
:1028E00029F0812F0E94781D0E949F1D802F0F903C
:1028F0000F900F900F900F90DF91CF911F910F913C
:10290000FF90EF90DF90CF900C940413802F0E94E3
:10291000CE13112309F4B8C2812F0E947E1D0F909F
:102920000F900F900F900F90DF91CF911F910F910B
:10293000FF90EF90DF90CF900C949F1D812F807FB0
:102940001F70803211F01295107F002319F00130B2
:1029500009F12BC0FF20A9F0EE2059F1F1E0812F01
:10296000EF1228C00F900F900F900F900F90DF91F3
:10297000CF911F910F91FF90EF90DF90CF900C942B
:10298000881DEE2021F021E0E21609F47DC20E94AC
:102990008B1D4DC0FF20E9F085E08E1508F474C250
:1029A0000E94621D812329F042C0FF20F1F1E11055
:1029B00015C0812F0F900F900F900F900F90DF9107
:1029C000CF911F910F91FF90EF90DF90CF900C94DB
:1029D000F61394E09E1508F457C229C0F6018581CC
:1029E00080FF13C08F708583E4CF003F09F489C155
:1029F00008F055C180E4800F803208F459C1FF20EF
:102A000009F4EAC1EE2009F49AC1802F0E94041350
:102A1000093309F0DAC1FFEF21EE84E0F1502040E4
:102A20008040E1F700C000002FC2E110D7C1812F24
:102A300059C1812F86958695837019F08130B9F040
:102A400023C2FF2019F0C801937002C080E090E01B
:102A50000F900F900F900F900F90DF91CF911F91DB
:102A60000F91FF90EF90DF90CF900C946E11FF20AC
:102A700019F0C801937002C080E090E00F900F90B1
:102A80000F900F900F90DF91CF911F910F91FF90BA
:102A9000EF90DF90CF900C949B11802FFF2019F0C6
:102AA0000E94971F02C00E94FF1F0F900F900F906F
:102AB0000F900F90DF91CF911F910F91FF90EF90AA
:102AC000DF90CF900C948420812F837009F070C028
:102AD000F110DAC1202F229526952770220F220FA0
:102AE000602F6F70862F90E0A0E0B0E06C017D0158
:102AF000022E04C0CC0CDD1CEE1CFF1C0A94D2F785
:102B000004FF12C08FE090E0A0E0B0E004C0880FA6
:102B1000991FAA1FBB1F2A95D2F7BC01CD01609552
:102B200070958095909503C060E070E0CB0116959C
:102B3000169513701230B1F040F56C297D298E295D
:102B40009F29113031F10F900F900F900F900F903F
:102B5000DF91CF911F910F91FF90EF90DF90CF9079
:102B60000C94B01B6C297D298E299F290F900F9002
:102B70000F900F900F90DF91CF911F910F91FF90C9
:102B8000EF90DF90CF900C94CA1B0E94B01BC7013E
:102B9000B6010F900F900F900F900F90DF91CF9193
:102BA0001F910F91FF90EF90DF90CF900C94961BA8
:102BB000FF2019F0812F817001C08695882309F4C8
:102BC00063C1202F229526952770220F220F602F98
:102BD0006F70862F90E0A0E0B0E06C017D01022EC6
:102BE00004C0CC0CDD1CEE1CFF1C0A94D2F704FFC1
:102BF00012C08FE090E0A0E0B0E004C0880F991F01
:102C0000AA1FBB1F2A95D2F7BC01CD016095709514
:102C10008095909503C060E070E0CB011695169505
:102C200013701230B1F040F56C297D298E299F294F
:102C3000113031F10F900F900F900F900F90DF91A6
:102C4000CF911F910F91FF90EF90DF90CF900C9458
:102C5000771C6C297D298E299F290F900F900F904A
:102C60000F900F90DF91CF911F910F91FF90EF90F8
:102C7000DF90CF900C94891C0E94771CC701B6018D
:102C80000F900F900F900F900F90DF91CF911F91A9
:102C90000F91FF90EF90DF90CF900C94651C023F56
:102CA00009F45EC008F449C0033F09F46CC0A7CE24
:102CB000902F9071E92E812F8F71FF2051F00E948B
:102CC000FE1B802FEE2019F08295807F73CE8F70CF
:102CD00071CE0E941F1C802FEE2019F08295807FFC
:102CE00001C08F700F900F900F900F900F90DF9199
:102CF000CF911F910F91FF90EF90DF90CF900C94A8
:102D0000FD13FF20A9F0E4E0EE1508F4BDC0812F0B
:102D10008F710F900F900F900F900F90DF91CF91C8
:102D20001F910F91FF90EF90DF90CF900C94441C77
:102D3000F5E0FE1508F4A8C0EACFFF2099F0812F36
:102D40008F710F900F900F900F900F90DF91CF9198
:102D50001F910F91FF90EF90DF90CF900C94FE1B8E
:102D6000FF2069F3812F8F710F900F900F900F90BC
:102D70000F90DF91CF911F910F91FF90EF90DF9017
:102D8000CF900C941F1CFF2089F0812F8F710F9022
:102D90000F900F900F900F90DF91CF911F910F9197
:102DA000FF90EF90DF90CF900C94E91B0F900F9065
:102DB0000F900F900F90DF91CF911F910F91FF9087
:102DC000EF90DF90CF900C94E41B033509F423CEF1
:102DD000073409F059C01FCEEE2021F2802F0F904A
:102DE0000F900F900F900F90DF91CF911F910F9147
:102DF000FF90EF90DF90CF900C94CE13412F4F7047
:102E0000602FC6010E940D1F0F900F900F900F9022
:102E10000F90DF91CF911F910F91FF90EF90DF9076
:102E2000CF900C94E61A01112FC0FF2069F10E9487
:102E300016142FEF80E792E0215080409040E1F798
:102E400000C000000F900F900F900F900F90DF9137
:102E5000CF911F910F91FF90EF90DF90CF900C9446
:102E6000AF1E412F4F70602FC6010F900F900F9033
:102E70000F900F90DF91CF911F910F91FF90EF90E6
:102E8000DF90CF900C94101F0F900F900F900F9029
:102E90000F90DF91CF911F910F91FF90EF90DF90F6
:102EA000CF9008951F93CF93DF9300D000D01F924F
:102EB000CDB7DEB7942F4983252F5A836B837C834C
:102EC0008D834C815D81452B31F02F3F31F481E0C2
:102ED0009F3F19F403C081E001C080E0182F1170FA
:102EE00080FD24C049815A816B817C818D810E9443
:102EF0009C1C292F22952F702C3030F42A3048F456
:102F00002250223068F013C02C3061F02F3051F085
:102F10000EC0803C28F0803E50F0815F833038F056
:102F200011E005C093FB112710F901C010E0812FBB
:102F30000F900F900F900F900F90DF91CF911F91F6
:102F40000895CF93DF9300D000D01F92CDB7DEB7A6
:102F50000F900F900F900F900F90DF91CF910895E9
:102F6000CF93DF9300D000D000D0CDB7DEB7269648
:102F70000FB6F894DEBF0FBECDBFDF91CF9108959D
:102F8000CF93DF93C091630280916402C817A1F0D0
:102F9000D0E0CE0166E070E00E94D526FC01EB593E
:102FA000FD4F4081518162817381848195810E94AE
:102FB000B0172196C770E8CFDF91CF910895409167
:102FC00095025091960260919702709198028091BB
:102FD000990290919A020C94B0171F93CF93DF93AC
:102FE00080919A0282958F7009F05CC0809197025F
:102FF000882309F457C02091630210916402C091A4
:103000009502D0919602A0919802B091990281E028
:10301000CF3F09F080E0482F211709F443C01097F3
:1030200021F0DF3F21F080E003C081E001C0842F68
:1030300030E080FD33C0C90166E070E00E94D52613
:10304000FC01EB59FD4F81818D1328C080818C13C9
:1030500025C08281811122C0838194818A1B9B0BB0
:10306000883C9105D8F480919A028F70806180939A
:103070009A02C90166E070E00E94D526FC01E6597B
:10308000FD4F90819F709061908385E992E00E944E
:103090001A14DF91CF911F910C94C0172F5F3F4FEF
:1030A0002770BACFDF91CF911F9108959F92AF9271
:1030B000BF92CF92DF92EF92FF920F931F93CF9325
:1030C000DF93CDB7DEB761970FB6F894DEBF0FBEC2
:1030D000CDBF8C0185E0F801DE011D9601900D92B7
:1030E0008A95E1F7F80140812181F280C380D48084
:1030F0009091950230919602609198027091990298
:103100006115710531F03F3F31F481E09F3F19F4C3
:1031100003C081E001C080E0F82FF1709F2E80FD98
:1031200059C185E9A82E82E0B82EE0909702F601F9
:10313000E61BF70BEE2009F4EDC080919A02582FA0
:10314000507FE83CF10508F0A7C0511156C0231389
:1031500013C0491311C0EF2CF1100EC08F708061A5
:1031600080939A020E94DF17C5010E941A14809171
:103170009A02F801858364C1C114D10431F02F3F54
:1031800031F481E04F3F19F403C081E001C080E0D9
:1031900080FD03C081E08F2502C080E090E0F82F21
:1031A000F170EF2E80FF1FC0E09163023091640246
:1031B000E31709F421C1F0E0CF0166E070E00E945E
:1031C000D526DC01AB59BD4F11968C911197281370
:1031D00007C08C91481304C012968C91F81203C05A
:1031E0003196E770E5CFEF2CFF2009F429C18091DB
:1031F0009A02816080939A0264C0231306C0491327
:1032000004C0F11002C0F801A9C04D872E87FF86C7
:103210007C2DD98AC88A522F6F2D89890E94521716
:103220008823A1F1FF2091F120919A02822F8295AB
:103230008F7090E0029774F08091950290919602C1
:1032400098878F831986DB86CA862C87CE010796DE
:103250000E941A1486E0F801A5E9B2E001900D92EF
:103260008A95E1F70E94ED170E94DF1712C023171D
:1032700051F14D872E87FF867C2DD98AC88A522F1F
:103280006F2D89890E94521781112CC0C8010E949C
:103290001A14EE24E394D4C05111E9CF7C2DD98ABD
:1032A000C88A522F6F2D89890E94A11785E992E063
:1032B0000E941A1486E0F50111928A95E9F70E949E
:1032C000DF17E12CBDC04913D4CFF110D2CFF801E4
:1032D0008583C8010E941A1486E0F50111928A952F
:1032E000E9F7AEC0FF2091F220919A02822F8295D9
:1032F0008F7090E002970CF4ADCF80919502909181
:1033000096029A8389831B82DD82CC822E83CE0132
:1033100001969ECFE83CF10508F04CC0EF2CFF2051
:1033200009F4B4CF231330C049132EC020919A0260
:1033300020FD21C0822F82958F70482F50E04115CB
:103340005105C9F0F80125834F30510541F08F5FD9
:10335000982F9295907F822F8F70892B8583C8013B
:103360000E941A1486E0F801A5E9B2E001900D92DE
:103370008A95E1F72CC086E0F801A5E9B2E001905A
:103380000D928A95E1F75CC04D872E87FF867C2DD4
:10339000D98AC88A522F6F2D89890E9452178111AC
:1033A00059CF80919A02816080939A02C8010E944D
:1033B0001A1446C07C2DD98AC88A522F6F2D89894C
:1033C0000E94A11786E0F50111928A95E9F70E9403
:1033D000DF1736C0FF2009F459CF4D872E87FF86AF
:1033E0007C2DD98AC88A522F6F2D89890E94521745
:1033F000882309F44BCF2ECF7C2DD98AC88A522F2F
:103400006F2D89890E949C1C292F22952F702230B4
:1034100028F49F7039F0811105C00BC0243028F4C6
:103420009F7049F4805E883020F0C8010E941A1411
:103430009E2CE92C05C0F8019581907F99F7F9CF72
:103440008E2D61960FB6F894DEBF0FBECDBFDF9113
:10345000CF911F910F91FF90EF90DF90CF90BF9091
:10346000AF909F900895CF93DF93CDB7DEB72C97A1
:103470000FB6F894DEBF0FBECDBF4F835887698764
:103480007A878B879C87CE0107960E9456188823DF
:10349000D1F09F8188852A853B85232B31F08F3F92
:1034A00031F481E09F3F19F403C081E001C080E066
:1034B00080FD6FC04F81588569857A858B859C8595
:1034C0000E94B01766C086E0FE013796DE011196B5
:1034D00001900D928A95E1F7FF81E8856A857B85E9
:1034E0006115710531F0EF3F31F481E0FF3F19F4D0
:1034F00003C081E001C080E080FD4BC08091640288
:1035000090E09C012F5F3F4F27703327409163026B
:1035100050E02417350709F443C0F983EA837D831B
:103520006C8366E070E00E94D526DC01AB59BD4F8C
:1035300096E0FE01319601900D929A95E1F7209365
:1035400064020E94C01725C090E066E070E00E940F
:10355000D5268B599D4F0E945618882371F1809172
:10356000630290E066E070E00E94D526FC01EB5912
:10357000FD4F4081518162817381848195810E94D8
:10358000B0178091630290E001968770992780932D
:10359000630280916302909164028913D5CF0DC0BC
:1035A0000E9416141092640210926302E5E9F2E0A0
:1035B00086E0DF011D928A95E9F72C960FB6F89404
:1035C000DEBF0FBECDBFDF91CF910895DF92EF92A6
:1035D000FF920F931F93CF93DF93FC01892B09F484
:1035E00088C0E12CF12CDD24D394EF012196849145
:1035F000853709F460C058F4843708F04EC0843031
:1036000008F068C08130D1F0823071F172C0883723
:1036100009F45BC050F4863709F453C0873709F0CA
:1036200068C08E2D0E94721D52C09CE7980F903783
:1036300008F05FC08F770E94CE134EC08F010E5FDF
:103640001F4FFE01849190E2980F983050F48770DC
:10365000FD2D01C0FF0F8A95EAF78F2F0E94781D7C
:1036600015C00E94041314C08F010E5F1F4FFE018E
:10367000849190E2980F983068F48770FD2D01C016
:10368000FF0F8A95EAF78F2F0E947E1D0E949F1DD3
:10369000E80122C00E94CE13FBCFCF010296FE01AB
:1036A000C491CC2361F0EFE9FFE03197F1F700C05E
:1036B0000000C150F6CFCF010296FE01F490EC015C
:1036C0000BC00E94621DE82E07C00E94751D0E945B
:1036D0009F1D02C00E9404138F2D882341F0EFE943
:1036E000FFE03197F1F700C000008150F6CFFE01F6
:1036F0007CCFDF91CF911F910F91FF90EF90DF90E2
:1037000008956093FB027093FC028093FD029093F6
:10371000FE020C94EE1D08956093FF027093000367
:1037200080930103909302030C94ED1D0F931F935C
:103730000091FF02109100032091010330910203D8
:10374000602B712B822B932B6093FF0270930003ED
:1037500080930103909302031F910F910C94ED1D30
:103760000F931F930091FF0210910003209101031A
:103770003091020360237123822393236093FF021D
:103780007093000380930103909302031F910F91A4
:103790000C94ED1D0F931F930091FF0210910003F5
:1037A000209101033091020360277127822793271C
:1037B0006093FF02709300038093010390930203D0
:1037C0001F910F910C94ED1D60E070E0CB010C9403
:1037D000811B0F931F9341E050E060E070E08A018D
:1037E0009B0104C0000F111F221F331F8A95D2F7BF
:1037F000C901B8011F910F910C94811B0F931F9366
:1038000041E050E060E070E004C0440F551F661FC7
:10381000771F8A95D2F78091FB029091FC02A091CC
:10382000FD02B091FE028A019B01082B192B2A2B65
:103830003B2BC901B8011F910F910C94811B0F9371
:103840001F9341E050E060E070E004C0440F551F5A
:10385000661F771F8A95D2F74095509560957095B1
:103860008091FB029091FC02A091FD02B091FE02BA
:103870008A019B01082319232A233B23C901B8018C
:103880001F910F910C94811B0F931F9341E050E007
:1038900060E070E004C0440F551F661F771F8A95D3
:1038A000D2F78091FB029091FC02A091FD02B091B1
:1038B000FE028A019B01082719272A273B27C901F5
:1038C000B8011F910F910C94811B0F931F930091CE
:1038D000FB021091FC022091FD023091FE02602B50
:1038E000712B822B932B1F910F910C94811B0F93A3
:1038F0001F930091FB021091FC022091FD02309178
:10390000FE0260237123822393231F910F910C9455
:10391000811B0F931F930091FB021091FC022091D9
:10392000FD023091FE0260277127822793271F91A5
:103930000F910C94811B08958F929F92AF92BF922A
:10394000DF92EF92FF920F931F93CF93DF9300D0FC
:1039500000D01F92CDB7DEB76B837C838D838A0145
:103960008C819D81892B31F01F3F31F481E04F3FE5
:1039700019F403C081E001C080E080FF03C080E053
:1039800090E054C08B81882309F43DC08090FB02F5
:103990009090FC02A090FD02B090FE028091FF0288
:1039A00090910003A0910103B0910203882A992A03
:1039B000AA2ABB2A2FE1E22EF12CD501C4010E2C3C
:1039C00004C0B695A795979587950A94D2F780FD80
:1039D00006C081E0E81AF10880F7D12C07C0DE2C80
:1039E000B8018E2D0E94E01E019799F3E12FF0E0BF
:1039F00093E0EE0FFF1F9A95E1F7E556FD4FE00FBC
:103A0000F11DD0820CC0E12FF0E083E0EE0FFF1F2C
:103A10008A95E1F7E556FD4FE00FF11DD08009834F
:103A20001A8369817A818D2D0E94E01E0F900F907C
:103A30000F900F900F90DF91CF911F910F91FF90FA
:103A4000EF90DF90BF90AF909F908F90089520915E
:103A5000120130911301F90132969FEF40E051912C
:103A6000851789F09F3F19F4511101C0942F4F5FC2
:103A70004630A9F79F3F39F0F901E90FF11D97FD95
:103A8000FA95828308950895E0911201F09113014F
:103A90009F012A5F3F4F9281891301C012823196A4
:103AA000E217F307C1F7089581E090E0E091120179
:103AB000F0911301E80FF91F1082019688309105EB
:103AC000A9F7089580910D03089590910D03892B16
:103AD00080930D030895809590910D038923809321
:103AE0000D03089580930D03089510920D0308951A
:103AF00090910C03892B80930C03089580959091ED
:103B00000C03892380930C03089510920C030895ED
:103B10008093030308951092030308958091120186
:103B200090911301FC0131969C01285F3F4F80E08A
:103B3000919191118F5FE217F307D1F70895E0910A
:103B40001201F091130180910D038083E091120125
:103B5000F0911301908180910C03892B80838091D7
:103B60000303882361F0E0911201F0911301908129
:103B7000892B80830E948E1D8111109203038091F6
:103B80001201909113010C940711909335018093C9
:103B9000340108958295982F9373292F220F220FB5
:103BA000982F9C7C96959695922B892F8575880FDA
:103BB0009A7A9695892B089508950895CF93DF9367
:103BC00000D000D01F92CDB7DEB70F900F900F90AE
:103BD0000F900F90DF91CF910895089508950C9460
:103BE000711280E0089580912303843021F11092B6
:103BF0000F0320E488E190E00FB6F894A895809335
:103C000060000FBE2093600083B7817F846083BF14
:103C100083B7816083BF7894889583B78E7F83BF95
:103C20000FB6F894A8958091600088618093600039
:103C3000109260000FBE0895CF930E94BC120E94A4
:103C4000AA060E94BD12C0E08C2F0E94D3078111EA
:103C500004C0CF5FCC30C1F701C081E0CF9108959F
:103C60001F920F920FB60F9211248F939F93AF93D1
:103C7000BF9380910F03811113C080911003909125
:103C80001103A0911203B09113034196A11DB11D20
:103C90008093100390931103A0931203B093130326
:103CA000BF91AF919F918F910F900FBE0F901F907A
:103CB000189582E084BD93E095BD9AEF97BD8093FF
:103CC0006E0008952FB7F89480911003909111031E
:103CD000A0911203B09113032FBF08952FB7F8944A
:103CE000609110037091110380911203909113035E
:103CF0002FBF08959C014FB7F894809110039091C5
:103D00001103A0911203B09113034FBF821B930BB9
:103D1000089578941F920F920FB60F9211248F93EB
:103D20009F93AF93BF938091100390911103A09143
:103D30001203B09113030196A11DB11D80931003CE
:103D400090931103A0931203B0931303BF91AF910B
:103D50009F918F910F900FBE0F901F9018950E940A
:103D6000CE0FF89487E797E79093010880930008B7
:103D700087E090EBDC0180932C0390932D03A093BC
:103D80002E03B0932F039CE088E10FB6F894A8951A
:103D9000809360000FBE90936000FFCFE92FF0E0AA
:103DA00093E0EE0FFF1F9A95E1F7E80FF11DE8553C
:103DB000FF4F8491982F92959F708F709770089500
:103DC000CF93C82FCB010E94CE1E292F30E054E0A4
:103DD000220F331F5A95E1F7282B203831051CF0AC
:103DE00080E090E018C0EC2FF0E023E0EE0FFF1F22
:103DF0002A95E1F79770E90FF11D34E0EE0FFF1FF0
:103E00003A95E1F78F70E80FF11DEE0FFF1FE050BC
:103E1000F84985919491CF91089580E090E00895BC
:103E200008958091160380FF0CC08091170190E0E7
:103E300065E070E00E94D5269595879595958795C4
:103E40002EC081FF0AC08091170190E065E070E00C
:103E50000E94D5269595879522C082FF08C0809143
:103E6000170190E065E070E00E94D52618C020910F
:103E700017032223D9F030911601231780F7809180
:103E8000170190E065E070E00E94D526622F70E097
:103E90000E94D526632F70E00E94E626CB01803871
:103EA000910538F4009739F481E005C085E090E091
:103EB00008958FE7089508958091160380FF08C044
:103EC0006091150170E0759567957595679523C0AC
:103ED00081FF06C06091150170E0759567951BC064
:103EE00082FF04C06091150170E012C06091170359
:103EF0006623A9F0209114016217A0F780911501A3
:103F000070E090E00E94D526622F70E00E94E626C5
:103F10006038710540F46115710519F406C061E05F
:103F200070E0862F08958FE7089581E00895803F1F
:103F300021F40E94111F819504C0813F29F40E9441
:103F4000111F80931A030895823F21F40E94111FCC
:103F5000819504C0833F29F40E94111F80931903A7
:103F60000895893F19F40E945C1F05C08A3F31F40F
:103F70000E945C1F819580931B0308958B3F21F461
:103F80000E945C1F819504C08C3F29F40E945C1F35
:103F900080931C030895843F21F48091180381606D
:103FA00017C0853F21F480911803826011C0863FBD
:103FB00021F48091180384600BC0873F21F4809125
:103FC0001803886005C0883F31F480911803806130
:103FD0008093180308958D3F21F48091160381602A
:103FE0000BC08E3F21F480911603826005C08F3F85
:103FF00029F4809116038460809316030895803F0E
:1040000039F480911A0387FF6CC010921A0369C0BB
:10401000813F29F480911A031816BCF362C0909175
:104020001903823F29F497FF5CC01092190359C00D
:10403000833F19F41916CCF354C0893F41F48091A1
:104040001B0318160CF04DC010921B034AC08A3F88
:1040500029F480911B0387FF44C0F6CF8B3F39F4CE
:1040600080911C0387FF3DC010921C033AC08C3F17
:1040700029F480911C031816BCF333C0843F21F44B
:10408000809118038E7F17C0853F21F4809118031B
:104090008D7F11C0863F21F4809118038B7F0BC068
:1040A000873F21F480911803877F05C0883F31F452
:1040B000809118038F7E8093180313C08D3F21F4E5
:1040C000809116038E7F0BC08E3F21F480911603E2
:1040D0008D7F05C08F3F29F4809116038B7F8093DD
:1040E00016038091190381110EC080911A0381116A
:1040F0000AC080911B03811106C080911C038111AD
:1041000002C010921703089580910E0383FF7EC0B2
:104110008CE494E00E947705809118031F928F939E
:1041200087E494E09F938F930E94100685E494E0C7
:104130000E94770580911903282F082E000C330B5D
:104140003F938F9382E494E09F938F930E94100695
:1041500080E494E00E94770580911A03282F082EAE
:10416000000C330B3F938F938DE394E09F938F93D9
:104170000E9410068BE394E00E94770580911B0358
:10418000282F082E000C330B3F938F9388E394E085
:104190009F938F930E94100686E394E00E94770518
:1041A00080911C03282F082E000C330B3F938F9314
:1041B00083E394E09F938F930E94100680E394E042
:1041C0000E947705809117031F928F938DE294E0F0
:1041D0009F938F930E9410068BE294E00E947705D4
:1041E000809116031F928F9388E294E09F938F93A0
:1041F0000E94100685E294E00E9477058DB79EB775
:104200004C960FB6F8949EBF0FBE8DBF88E193E029
:104210000E9450110E94621E909315038093140314
:1042200008951F93CF93DF9380911403909115030A
:104230000E947A1EFC0120911703222321F0809115
:10424000180190E007C08091190190E06AE070E0E9
:104250000E94D526E817F90708F485C08091190354
:10426000C0911A03D0911B0310911C03811107C048
:10427000C11175C0D11173C0111171C074C02F3F2D
:1042800019F02F5F20931703181624F40E94111FB2
:10429000809319038091190387FF05C00E94111FA5
:1042A0008195809319031C1624F40E94111F80939A
:1042B0001A0380911A0387FF05C00E94111F819580
:1042C00080931A0360911903662331F1C0911A0398
:1042D000CC2311F1062E000C770B880B990B0E9452
:1042E000D42523E333E343E35FE30E9438260E94AF
:1042F0009C25609319036C2FCC0F770B880B990BBF
:104300000E94D42523E333E343E35FE30E9438268E
:104310000E949C2560931A031D1624F40E945C1FC2
:1043200080931B0380911B0387FF05C00E945C1FC5
:10433000819580931B03111624F40E945C1F8093C7
:104340001C0380911C0387FF05C00E945C1F8195A0
:1043500080931C03DF91CF911F910C9484202F3FF9
:1043600009F08FCFA0CFDF91CF911F910895E8E1A1
:10437000F3E085E0DF011D928A95E9F710921703BB
:104380001092160308958091180308958FE696E021
:104390000E9477051F9281E08F931F9285E08F9393
:1043A00081E296E09F938F930E9410060F900F90EA
:1043B0000F900F900F900F9008958330E9F128F43B
:1043C000813061F0823009F10895853009F462C0CE
:1043D00008F449C0863009F474C008958091190129
:1043E000262F30E0280F311D2F3F310524F4680FB0
:1043F0006093190103C08FEF809319018091190117
:104400001F928F938AE595E072C080911801262F44
:1044100030E0280F311D2F3F310524F4680F6093E1
:10442000180103C08FEF80931801809118011F922B
:104430008F9388E495E05BC080911701262F30E0D0
:10444000280F311D2F3F310524F4680F60931701A9
:1044500003C08FEF80931701809117011F928F93F4
:1044600085E395E044C080911601262F30E0280FA7
:10447000311D2F3F310524F4680F6093160103C0EE
:104480008FEF80931601809116011F928F9380E227
:1044900095E02DC080911501262F30E0280F311DA9
:1044A0002F3F310524F4680F6093150103C08FEF8F
:1044B00080931501809115011F928F9387E095E0FD
:1044C00016C080911401262F30E0280F311D2F3F98
:1044D000310524F4680F6093140103C08FEF8093BB
:1044E0001401809114011F928F938CEE94E09F939E
:1044F0008F930E9410060F900F900F900F900895C9
:10450000833081F128F4813059F08230D1F0089560
:10451000853009F449C0B8F1863009F456C00895D1
:1045200080911901681720F4861B8093190102C03D
:1045300010921901809119011F928F938DED94E0D3
:1045400054C080911801681720F4861B80931801CD
:1045500002C010921801809118011F928F938BEC6A
:1045600094E043C080911701681720F4861B809364
:10457000170102C010921701809117011F928F93AB
:1045800088EB94E032C080911601681720F4861BF6
:104590008093160102C010921601809116011F929D
:1045A0008F9383EA94E021C080911501681720F46D
:1045B000861B8093150102C0109215018091150190
:1045C0001F928F938AE894E010C0809114016817BD
:1045D00020F4861B8093140102C010921401809174
:1045E00014011F928F938FE694E09F938F930E9404
:1045F00010060F900F900F900F900895CF93C82F33
:104600001F928F9384E797E09F938F930E941006E9
:1046100081E090E0A0E0B0E0BC01CD0104C0660FF5
:10462000771F881F991FCA95D2F70E948C1B0F9085
:104630000F900F900F90CF910C941614CF93873258
:1046400088F58E3108F00BC18E3009F487C0D8F49C
:10465000873009F460C08B3009F44FC0863009F010
:1046600002C180910E03817F8E7F80930E0389E7C4
:1046700097E00E9477058DE39AE00E94770581E03C
:1046800080931E0346C0863109F4B0C020F4803107
:1046900009F47AC0E8C0893109F491C08B3109F47A
:1046A00049C0E1C0883349F150F4893209F4D5C0DA
:1046B000853309F4D2C0873209F0D5C0CEC0833427
:1046C00009F4CBC028F48A3308F4CDC08953C8C09C
:1046D000883409F0C8C00E9416148CE29AE00E9447
:1046E00077052FEF83ED90E3215080409040E1F774
:1046F00000C000000E94AF1E0CC080EA97E041C0DD
:1047000083E19AE00E94770580910E038160809397
:104710000E03C1E0ADC080910E03C82FC17080FFB1
:10472000EFCF8FE19AE00E94770580910E03817FA1
:104730008E7F3FC090910E0391FBCC27C0F981E0A2
:10474000C827892FC0FB81F980930E03CC2319F071
:1047500086E09AE029C088EF99E013C090910E039B
:1047600092FBCC27C0F981E0C827892FC0FB82F9D2
:1047700080930E03CC2319F089EE99E015C089EDE2
:1047800099E00E947705C5CF90910E0393FBCC274B
:10479000C0F981E0C827892FC0FB83F980930E03FD
:1047A000CC2351F08DEC99E00E94770580910E03A7
:1047B000816080930E035CC080EC99E0E2CF81EBD6
:1047C00099E00E94770582E899E00E94770585E3E9
:1047D00099E00E9477058FE099E00E9477058AECC6
:1047E00098E00E9477058EE998E0CBCF80E998E0C9
:1047F0000E9477050E94FB101F928F9386E798E036
:104800009F938F930E941006809111011F928F93A6
:104810008FE598E09F938F930E94100680914F023E
:104820001F928F938CE498E09F938F930E941006C1
:104830000E946E1E9F938F937F936F9385E398E002
:104840009F938F930E9410068DB79EB742960FB626
:10485000F8949EBF0FBE8DBF5CCF80E001C08D512C
:104860000E94FE2256CF83E398E00E947705C0E0C5
:104870008C2FCF91089580E008950C943B24CF9322
:10488000C82F80911E03813091F020F0823009F40E
:1048900053C04AC1E0911201F0911301808182322C
:1048A00089F0803479F0803809F040C10BC0E09184
:1048B0001201F09113018081823221F0803411F0D5
:1048C000803861F48C2F0E943D24811104C08C2F0C
:1048D0000E941E232FC081E090E02CC08C2F0E94EC
:1048E0003B24811126C0C431E1F070F4CB3081F05B
:1048F000C031D1F40E94C6218CE697E00E94770572
:1049000082E080931E0315C0C93259F0C83361F4A8
:1049100089E797E00E94770580E797E00E94770596
:1049200008C010921E0304C18AE697E00E94770532
:10493000FFC081E08170FEC0C43228F5CE3108F09E
:10494000C1C0CB30A1F1D0F4C73009F0D3C08EE1A3
:104950008093190182E3809318018AE08093170104
:1049600084E18093160188E08093150188E28093AA
:10497000140180E196E00E947705BFC0C33149F180
:10498000C431C1F0B7C0CB3409F4A9C028F4C9328E
:1049900089F0C83361F0AEC0C13509F49EC0C2359C
:1049A00009F499C0CE3409F0A5C06AE09EC00E9407
:1049B000C621A3C080911D03882319F010921D0306
:1049C0009CC08DE196E00E94770581E080931E03F4
:1049D000B1C087EF95E00E94770585EE95E00E94D3
:1049E0007705809119011F928F9382EE95E09F9336
:1049F0008F930E94100680EE95E00E9477058EEC62
:104A000095E00E947705809118011F928F938BEC9F
:104A100095E09F938F930E94100689EC95E00E9489
:104A200077058AEB95E00E947705809117011F9228
:104A30008F9387EB95E09F938F930E94100685EBF1
:104A400095E00E94770584EA95E00E9477058091C1
:104A500016011F928F9381EA95E09F938F930E9496
:104A600010068FE995E00E9477058AE895E00E949C
:104A70007705809115011F928F9387E895E09F93AA
:104A80008F930E94100685E895E00E9477058EE6D8
:104A900095E00E947705809114011F928F938BE619
:104AA00095E09F938F930E94100689E695E00E94FF
:104AB00077058DB79EB748960FB6F8949EBF0FBE88
:104AC0008DBF1BC0CE51EC2FF0E0E65DFE4F808124
:104AD00080931D0312C061E003C061E006C06AE07C
:104AE00080911D030E94DD2108C080911D030E945A
:104AF000802203C08EE096E013C080911D038823BE
:104B000069F01F928F9388E096E09F938F930E94A5
:104B100010060F900F900F900F9004C085E096E064
:104B20000E94770581E006C010921E0380E002C05B
:104B300080E000CFCF9108950E94A3256894B11121
:104B40000C94322608950E94172688F09F5798F0FB
:104B5000B92F9927B751B0F0E1F0660F771F881F82
:104B6000991F1AF0BA95C9F714C0B13091F00E949C
:104B70003126B1E008950C943126672F782F8827CD
:104B8000B85F39F0B93FCCF3869577956795B395C3
:104B9000D9F73EF490958095709561957F4F8F4F32
:104BA0009F4F0895E89409C097FB3EF49095809537
:104BB000709561957F4F8F4F9F4F9923A9F0F92FE3
:104BC00096E9BB279395F695879577956795B79561
:104BD000F111F8CFFAF4BB0F11F460FF1BC06F5F47
:104BE0007F4F8F4F9F4F16C0882311F096E911C059
:104BF000772321F09EE8872F762F05C0662371F07A
:104C000096E8862F70E060E02AF09A95660F771F8D
:104C1000881FDAF7880F9695879597F9089557FDBD
:104C20009058440F551F59F05F3F71F04795880F1A
:104C300097FB991F61F09F3F79F0879508951216B1
:104C400013061406551FF2CF4695F1DF08C016165D
:104C500017061806991FF1CF86957105610508940E
:104C60000895E894BB2766277727CB0197F9089525
:104C70000E944A260C94C4260E94B62638F00E9450
:104C8000BD2620F0952311F00C94AD260C94B3268C
:104C90000C9432260E940F2678F39923C9F35523EA
:104CA000B9F3950F50E0551FAA27EE27FF27BB2722
:104CB00000240894679520F4E20FF31FB41F0A1E26
:104CC000220F331F441FAA1F6695A9F7779530F46A
:104CD000F30FB41F0A1E121E08F46395330F441F0E
:104CE000AA1F221F769599F7879520F4B40F0A1E04
:104CF000121E631F440FAA1F221F331F8695A9F798
:104D0000862F712D602D11249F5750409AF0F1F09D
:104D100088234AF0EE0FFF1FBB1F661F771F881FF7
:104D200091505040A9F79E3F510580F00C94AD265C
:104D30000C9432265F3FE4F3983ED4F38695779542
:104D40006795B795F795E7959F5FC1F7FE2B880F9D
:104D5000911D9695879597F9089597F99F6780E833
:104D600070E060E008959FEF80EC089500240A94BD
:104D70001616170618060906089500240A94121636
:104D80001306140605060895092E0394000C11F469
:104D9000882352F0BB0F40F4BF2B11F460FF04C016
:104DA0006F5F7F4F8F4F9F4F08950024552704C09A
:104DB000080E591F880F991F009729F0769567955F
:104DC000B8F37105B9F7802D952F089597FB072E3D
:104DD00016F4009407D077FD09D00E94002707FC45
:104DE00005D03EF4909581959F4F089570956195FB
:104DF0007F4F0895EE0FFF1F0590F491E02D099469
:104E0000AA1BBB1B51E107C0AA1FBB1FA617B707F0
:104E100010F0A61BB70B881F991F5A95A9F780950C
:0C4E20009095BC01CD010895F894FFCFDF
:104E2C000546010000FFCE08700941090509D108AB
:104E3C00010104032808140A321E407F2291031238
:104E4C0003F0029C02B502CE020001020304050627
:044E5C00070809003A
:106800000000000000000000040005000600070072
:10681000080009000A000B000C000D000E000F001C
:1068200010001100120013001400150016001700CC
:10683000180019001A001B001C001D001E001F007C
:10684000200021002200230024002500260027002C
:10685000280000002A002B002C002D002E002F0005
:1068600030003100000033003400290036003700CA
:106870003800E00000000000000000000000000000
:106880000000000000000000000000000000000008
:106890000000E944E2444B00EA4400004E004F008F
:1068A0005000510052003500310054005500560090
:1068B000580059005A005B005C005D005E005F00FC
:1068C00060006100620063000000F1A15700000059
:1068D00000000000000000000000000000000000B8
:1068E00000000000000000000000000000000000A8
:1068F000E200E1000000E300E600E5000000000027
:106900000100010001000100EA4401000601E24427
:106910000100010001005500460054004A004B00F0
:10692000560057004700480031000100E9440100CB
:106930000100190101001B0101001D013A003B008B
:106940003C003D003E003F0040004100420043004B
:10695000010001004C0039000100440045005200D4
:1069600049000100010050004F0035004D004E006D
:1069700051000100010001000100010001000100BF
:1069800001000100010001000100010001000100FF
:1069900001000100010001000100010001004D00A3
:1069A0004A004E004B0053000100010001000100AD
:1069B00001000100010001000100010001000100CF
:1069C00001000100010001000100010001000100BF
:1069D00001000100010001000100010001000100AF
:1069E000010001000100010001000100010001009F
:1069F000010001000100010001000100010001008F
:00000001FF
